:020000020000FC
:100000003FC011C01AC031C037C018951895189557
:10001000189518951895189531C018951895189534
:10002000189518951895FFB6849B14C02AE0C20E47
:1000300020E0D21E1061FFBE1895FFB6849B7CC0E5
:100040002AE0C21A20E0D20A10F4DD24CC24106188
:10005000FFBE189513FD03C01460FFBE1895126013
:10006000FFBE18951560FFBE1895FFB61160019789
:1000700009F41260FFBE189596981895969A1895EF
:1000800000E806BD002706BD0FED0DBF8D9A9598BF
:100090008E9A96988A98929A8B98939A8C98949A1A
:1000A00011279198899A9098889A0FEF07BB92D060
:1000B00006E905BD00E004BD0BE40BBD00E00ABD90
:1000C00000E709BD00E808BD90E08AE049D059D0BA
:1000D00012D00FE205BF00EC0BBF789488950000AA
:1000E00011FD09D012FD14D010FD24D014FD20D034
:1000F00015FD22D0F3CF1D7F959800270CBF969851
:1001000000E00FBD08E10EBD00E009BF177F0895B4
:100110001B7F959A9D2D8C2D00E00DBD0CBD00E040
:100120000FBD0BE10EBD08E609BF969A186025C009
:100130001F7E27C01E7F21C01F7D00E40EBBF894E8
:10014000CDBAE29AE19A7894E199FECF01E40EBB30
:10015000F894DDBAE29AE19A7894E199FECF089595
:1001600000E40EBB01E00CBBCDB201E40EBB01E02C
:100170000CBBDDB200E00EBB08950AEC082E192E70
:1001800003C00AE80C2C1D2C909808BB8ED0A3D07D
:10019000909AFF27ECE322240E161F0620F00E1A79
:1001A0001F0A2394F9CF05D00AE308BB7ED093D071
:1001B000202C11240AE0201618F0201A1394FBCFEB
:1001C00000E3010D08BB71D086D000E3020D08BB2F
:1001D0006CD081C074D0909808E308BB66D072D010
:1001E00064D076D062D074D008E008BB5ED073D003
:1001F00001E008BB5AD063D006E008BB56D06BD0F4
:1002000000E108BB52D067D002E008BB4ED05DD001
:100210000FE008BB4AD05FD0909AF2E0E2E606D049
:100220000AEF4AD00A95E9F7F2E0EAE7909800E889
:1002300008BB3BD0909AFF93EF934DD0EF91FF9185
:10024000C8953196002061F00AE0001631F49098CC
:1002500000EC08BB2AD0909AEECF08BA26D0EBCF9C
:1002600037C054696D657220415474696E793233B8
:10027000313320444734464143004D61782E746940
:100280006D653D2030303A3030207365636F6E64A9
:10029000730A5265737474696D653D2030303A306D
:1002A00030207365636F6E647300919A00000000E4
:1002B0000000000091980895F8E1E8E610C0FAE027
:1002C000EAEF0DC0FAE0E0E00AC0F3E0EFEF07C0AC
:1002D000F0E0ECE304C0F0E0E7E10000000031975B
:0402E000F1F7089595
:00000001FF
